:020000040000FA
:0400000004303A2866
:08000800A000030EA100831209
:100010008B1C32288B1031181428B11C3228643004
:10002000010203183128182800001628172818285C
:1000300019281A281B281C281D281E281F283110A3
:10004000B114A810031005190314AA0DA90DA80DC9
:10005000B00B322831152A08AF002908AE00280855
:10006000AD00B11081010B11210E8300A00E200EF6
:02007000090085
:0C007400203084008001840A6030040207
:10008000031C3C281230B00077218316FF23900018
:10009000831283160C308505870183128501870141
:1000A000073099000030831691009F008312C830FA
:1000B00083168100831231309000003083168C004B
:1000C000831210308B00D12181018E018F010B1121
:1000D0008B100B108C018B177B2031199120B30BE7
:1000E0007928031085190314B90DF030390203196A
:1000F000FA20D2216C286400311808000B1D08007A
:100100000B11B11031141230B000051D8C283214BF
:10011000831601138312080032108316011783120D
:10012000080031110130B7008B13203037078316D8
:100130009B001C141A088312A400A500C030A50659
:100140001030370783169B001C141A088312A30073
:100150000030370783169B001C141A088312A20074
:100160008B17321CB92822090339A200A309A4095C
:10017000A50922082D02031DF42823082E02031DC1
:10018000F42824082F02031DDA2801303702031D4A
:10019000CC283D143E14852102303702031DD3289C
:1001A000BD143E14912103303702031DDA283D159A
:1001B0003E149D2125082F02031DF428013037022B
:1001C000031DE5283D103E14A92102303702031D0E
:1001D000EC28BD103E14AA2103303702031DF3287A
:1001E0003D113E14AB21F428B70A0430370203183E
:1001F000080094280130B600B300B400B500B70081
:1002000085018701B113C0217B20B30B272903107F
:1002100085190314B90DF030390203194E29B41FA2
:100220008501B41F8701B40B2729B50B272902309C
:10023000B500013037020319AC210230370203192F
:10024000B121033037020319BB21FA30B400311D4C
:1002500004293111321C31292D090339AD00AE09B1
:10026000AF092F1CB1132F1C0429B11B04292E1810
:100270000429B1178B1320303707BB002F08BA00B1
:10028000642110303707BB002E08BA00642100300B
:100290003707BB002D08BA0064218B17C3218501E5
:1002A0008701B70AB60104303702031C0429C001D4
:1002B0000800D12108003E1C08003E101030BB0091
:1002C0003D08BA00642108008B133A0883161C15F8
:1002D0009A003B089B0055309D00AA309D009C145D
:1002E00064009C1870291C1183128B170800831658
:1002F00020309B001C141A088312C2000130C21B5C
:10030000C200C2080319C200080085160512851034
:100310000510C001C0148E018F010C104208C100ED
:1003200008008516051285100510C00140158E01C4
:100330008F010C104208C1000800851205128514B7
:100340000510C001C0158E018F010C104208C100BC
:100350000800080008000800380903398500B800C3
:100360000800C00A38093339B800C01C0339C01866
:10037000303985000800380930398500B800080098
:10038000B801B8140800B80101303702031DCA29AA
:10039000B814381602303702031DD0290000B816F1
:1003A000080008000C1C08000C10C10B08004208D3
:1003B000C1008501C018051440198514C01905161F
:0E03C000C0018E018F010C104208C100080020
:084000000300030006000000AC
:02400E00CC01E3
:10420000010003000300030003000200020002009B
:1042100002000000000000000000FF00FF00FF009F
:10422000000000000000000000000000000000008E
:104230000000C000C000C000C000FF00FF00FF0081
:104240000100C300F300CF00FF00C300F300CF0064
:10425000FF00C300F300CF00FF00FF00FF00FF00DE
:10426000FF00FF00FF00FF00FF00FF00FF00FF0056
:10427000FF00FF00FF00FF00FF00FF00FF00FF0046
:10428000FF00FF00FF00FF00FF00FF00FF00FF0036
:10429000FF00FF00FF00FF00FF00FF00FF00FF0026
:1042A000FF00FF00FF00FF00FF00FF00FF00FF0016
:1042B000FF00FF00FF00FF00FF00FF00FF00FF0006
:1042C000FF00FF00FF00FF00FF00FF00FF00FF00F6
:1042D000FF00FF00FF00FF00FF00FF00FF00FF00E6
:1042E000FF00FF00FF00FF00FF00FF00FF00FF00D6
:1042F000FF00FF00FF00FF00FF00FF00FF00AA001B
:00000001FF
